:100000000C94E7030C940F040C940F040C940F044D
:100010000C940F040C940F040C940F040C940F0414
:100020000C940F040C940F040C940F040C94F41E05
:100030000C940F040C940F040C940F040C940F04F4
:100040000C94CC200C940F040C940F040C940F040B
:100050000C940F040C940F040C940F040C940F04D4
:100060000C940F040C940F04401AFFFFFFFFFFFFD6
:10007000FFFF0000000000000000300080C09F87EC
:10008000F0F8780081E0B3CF81EC7801C1E0A1CF36
:1000900003C67801C1F0A1EF03C27803E1F0A1EF3C
:1000A00003C27803E178A1EF03C27802E178A1EFFF
:1000B00003C27806F13CA1EFE3C67804F13CA1EF5E
:1000C00003FC7804791EA1EF03C6780FF91EA1EF97
:1000D00003C27808790FA1EF03C278083D0FA1EFA2
:1000E00003C278183D07A1CF03C27C103D07B3CFF0
:1000F00083C23FD019031F87F9820000000000006F
:100100000000FFFFFFFFFFFFFFFF000000000000F7
:100110000000A6C66AECE66E66CEAAAA8A4A8AAA39
:100120008AA8AAAEEA4ACAEC8EAC4AAA2A4A8AAA85
:100130008AA84ECAE4ECEEAAEACE0404F0F0F0F08D
:100140000404F07070F00404F030F0F00404F0F0F7
:1001500070F00404F07030F00404F0E0E0F0040407
:10016000F0C0F0F00404F0F0E0F00404F0E0C0F0BF
:10017000040490F0F0F00404D0D0F0F00404B0F0E7
:10018000F0F0040490B0F0F00404F0F0F0900404F7
:10019000F0F0B0B00404F0F0F0D00404F0F0D0902F
:1001A00004041070F0F00404101070F004041070D7
:1001B00030F00404105070F00404C0E0E0F00404D7
:1001C00080C0C0F0040480A0E0F0040480E0C0F02F
:1001D0000404F07070300404F03030100404F07047
:1001E00050100404F03070100404F0E0E0C0040487
:1001F000F0C0C0800404F0E0A0800404F0C0E080FF
:1002000004041030F030040430F0301004041030D6
:1002100070300404307030100404C0F0C080040456
:1002200080C0F0C00404C0E0C080040480C0E0C00E
:1002300004044040E0F00404202070F00404004076
:10024000E0F00404002070F00404F0E040400404F6
:10025000F07020200404F0E040000404F07020005E
:100260000404D0F0F0B00404B0F0F0D0040490D056
:10027000F0B00404D0F0B0900404F070E0F0040496
:10028000F0E070F00404F03060F00404F060C0F0BE
:10029000040460D0B0600606483078304800060696
:1002A000483078304884060668944488A458060686
:1002B00010449024882006068420084010840606F6
:1002C000100080040020040360F060150C000000A2
:1002D000000000000000000000000008400018E0DE
:1002E0000078E00038C00038E00078F104F8FFFF43
:1002F000F8150C0000000000000000800001809054
:1003000001C8FC03C8FE07D8F00FF8E007F8C003E7
:10031000F8F807F8FFFFF8150C003FF80009F8009F
:1003200000F80000B8020038760018FF0038FFC05F
:10033000B8FF81F8FF01F8FF80F8FFFFF8150C0700
:10034000FFF803FFF803FD7801785880501880000B
:1003500008800018D00008F40018FD03F8FF27F803
:10036000FFFFF8150C0000000000000000088000EE
:1003700018C80008FED808FFFC08FFF008FFA00816
:10038000FF0018FF80F8FFFFF8150C03789803D0E2
:100390000801C0188080088000088007C0C00FE8EE
:1003A000E01FE8C0F878E073387DE7983F8FC81504
:1003B0000C00000000000000450081FF80C7FFC066
:1003C000E3FFE0C1FFC0F09380F80000FC0000FEF6
:1003D0000008FEFFF8150C07C03807E01807801862
:1003E000030008038000030400810400C00C00E047
:1003F0000E00F01E00E0FF80FFFFF8150C00F03843
:1004000000600838C008E0C000C183C08187408315
:100410000FE0021BE0800FB0901FF0D03EF0FFFF16
:10042000F8150C01E03800F018487808FC3F88FC0B
:100430003FC0F87F80F07F00F0F600D040089000C9
:1004400018800078FFFFF8596F646127730020203F
:100450002020596F646127730020202020596F6489
:100460006127730003053F213F0A100A1208120E8C
:100470001C0E0C1E0C141A14161F161E131E1E1B07
:100480001E1E1F1E3F213F3A2F3A173D173F213FA7
:10049000181F02040A041F0E04040E1F0A1F0A0E6E
:1004A0000E1F04110E2E252E2F2A2E262929021F5B
:1004B00002081F08150E04040E150E15151B151B3A
:1004C000040604040C040000000017000300031FCE
:1004D0000A1F16371A1904130A153A000300000EF2
:1004E00011110E000A040A040E0400300004040472
:1004F0000010001804031F111F121F101D151711E3
:10050000151F07041F17151D1F151D01011F1F159E
:100510001F17151F000A00003200040A110A0A0AF8
:10052000110A040115020E11171E051E1F150A0ED1
:10053000110A1F110E1F15111F05010E111D1F0499
:100540001F111F1108100F1F041B1F10101F061F63
:100550001E040F0E110E1F09060E112E1F051A1272
:100560001509011F011F101F0F180F1F0C1F1B045F
:100570001B031C03191513001F11030418111F007E
:100580000201022020200001020C121E1F120C0C7E
:1005900012120C121F0C1A14041E05242A1E1F020C
:1005A0001C141D1020201D1F0814111F101E041ED6
:1005B0001E021C0C120C3E0A040C123E1E040214F5
:1005C000160A020F120E101E0E100E1E081E120C1E
:1005D0001226281E322A26041E21001F00211E0476
:1005E0000102013F213F0A4E6F2053442063617294
:1005F00064206F720A6E6F204C4F414445522E4862
:1006000045580A0A153A45786974001D20466C6100
:100610007368696E670A20206C6F616465722E2EA4
:100620002E0A0A444F4E2754205455524E204F460E
:100630004621004E4F20424154544552590A0A5017
:100640004C454153450A5455524E204F46460017DB
:100650007361766500166261636B0015747970656D
:10066000000A0A0A153A6F6B617920163A656469C7
:100670007400596F7520656E74657265640A005464
:100680000A03E181867F3E186D830F0F0E0183867A
:100690006033186DC3198F1803C38E6033186DE370
:1006A00030CF1803C39E603630CDE360CF3006C72D
:1006B0009E7E3E30CDB360CF300CC6F6603330D96D
:1006C000B660CF33CFCCF66061B0DB1E60CF30D8E0
:1006D0006CE6C061B0DB1E618F19986CC6C063B157
:1006E0009B0E330F0FB078C6FF7E1F1B061E0F1721
:1006F000534400161378001613140015102000152B
:10070000201000000005008930080238024978688E
:100710001400004500680100000500680138010070
:10072000000500380168010000F6E8DBCFC3B8AE71
:10073000A49B928A827B746E68625C57524E4945D4
:10074000413E3A3734312E2C29272523211F1D1CE9
:100750001A1917161514131211100F0E0D0C0B0A7F
:100760000908070668076C070101F7030101FF0389
:1007700000000000240027002A00000000002500DF
:1007800028002B000000000023002600290004049C
:100790000404040404040202020202020303030329
:1007A0000303010204081020408001020408102005
:1007B00001020408102000000007000201000003ED
:1007C00004060000000000000000B304AC04112483
:1007D0001FBECFEFD8E0DEBFCDBF12E0A0E0B1E09A
:1007E000E2E8F1E502C005900D92A235B107D9F714
:1007F00016E0A2E5B2E001C01D92A038B107E1F712
:1008000017E0CCECD7E004C02297FE010E947928C3
:10081000CA3CD107C9F70E9444230C94B4280C9415
:100820000000A0E0B0E0E7E1F4E00C948528EC01E2
:10083000A880B980CA80DB80A114B104C104D104AE
:1008400041F484E2A82E89EDB82E8BE5C82E87E00E
:10085000D82EC601B5012DE133EF41E050E00E94F2
:100860005C2827EA31E440E050E00E94E8277B0161
:100870008C01C601B5012DE133EF41E050E00E944B
:100880005C28CA01B9012CEE34EF4FEF5FEF0E94F4
:10089000E8276E0D7F1D801F911F97FF04C06150D8
:1008A000704080409048688379838A839B839B0152
:1008B000AC015F77B901CA01CDB7DEB7EAE00C94AD
:1008C000A1280E941104089588ED91E00E9411046E
:1008D00008956093D8017093D9018093DA019093C1
:1008E000DB010895FB01DC0102C001900D92415033
:1008F0005040D8F70895FB01DC018D9101908019DB
:100900000110D9F3990B0895FB01DC0101900D92C0
:100910000020E1F7089581309105A1F46F5F7F4FCA
:10092000D1F410921503109214038DE492E0909389
:100930001303809312038AE493E060E071E00E9465
:10094000B1250895892B39F46F5F7F4F21F48AE434
:1009500093E00E94E425089580E090E06FEF7FEF40
:100960000E948B04089581E090E06FEF7FEF0E947A
:100970008B0408958F929F92AF92BF92CF92DF9295
:10098000EF92FF920F931F937C01162F57E7852E4E
:1009900052E0952E49EFA42E41E0B42E6C0134E0D4
:1009A000CC0CDD1C3A95E1F7CA0CDB1CC40160E0FD
:1009B000F601448520E0012F0E94491AC40161E03C
:1009C000F601408120E00E94491AF6012085219518
:1009D000C40162E042850E94491A94E0EE0CFF1CBB
:1009E0009A95E1F7F60124812A53C40163E0468118
:1009F0000E94491AAE0CBF1CC401F5016281F601C8
:100A00004685212F0E94AE1A1F910F91FF90EF9003
:100A1000DF90CF90BF90AF909F908F900895EF920E
:100A2000FF920F931F93CF93DF9300E010E0EE242B
:100A300021C08881882389F090E001979C01220FD2
:100A4000331F280F391F220F331F265C3E4F82E1D0
:100A500093E06F2D4E2D0E94DD122C9684E0F80E4F
:100A600084E5F81631F70F5F1F4F84E0E80E80E34E
:100A7000E81629F0E801CD59DC4FFF24DACFDF91E9
:100A8000CF911F910F91FF90EF90089588E090E033
:100A9000909359038093580310925B0310925A036A
:100AA0008AE080935C0380935D038FEF9FEF9093C8
:100AB00062048093610410926003109260041092AB
:100AC0005F0484EF91E090935F0380935E038AE478
:100AD00093E061E071E00E94CB25089510925203EB
:100AE0001092510383E080935503109262038AE4CD
:100AF00093E069E071E00E94CB25089520915103B5
:100B000030915203809153039091540382179307BD
:100B100024F4309354032093530310921B03109238
:100B20001C0382E193E065E171E00E94AF246091D3
:100B30005103709152036A30710514F48EE001C0C4
:100B40008CE06436710514F420E001C022E093E0EB
:100B5000683E790714F490E001C092E0821B891B83
:100B600080931B0386E080931C0382E193E04AE0BC
:100B700050E00E949C2460915303709154036A30AA
:100B8000710514F482E401C080E46436710514F444
:100B900020E001C022E093E0683E790714F490E081
:100BA00001C092E0821B891B80931B0386E0809327
:100BB0001C0382E193E04AE050E00E949C2482E121
:100BC00093E06AE04DE028E630E00E94DD121092EA
:100BD0001B038AE280931C0382E193E069E271E0E7
:100BE0000E94AF248CE592E064E00E94730F88239A
:100BF00051F08AE493E06EE371E00E94CB2587E731
:100C000092E00E94181F8CE592E066E00E94730F4C
:100C1000882341F082E592E067E474E048E650E022
:100C20000E946D1808950F93809161049091620461
:100C30002FEF8F3F920709F44FC001979093620402
:100C40008093610482E193E060E00E94C30F82E13F
:100C500093E061E143E122E307E00E94C01082E1FA
:100C600093E061E00E94C30F82E180931B0384E163
:100C700080931C036091550370E06150704082E1E5
:100C800093E04AE050E00E949C248AE180931B0399
:100C900082E193E066E471E00E94AF2480916104F8
:100CA00090916204892BC1F48FEF9FEF90936204BF
:100CB000809361048091550381508093550388236C
:100CC00029F48AE493E061E571E004C08AE493E0EA
:100CD0006AE571E00E94CB250F9108950F938091F2
:100CE0006003813009F06DC080915F0490916004D1
:100CF00001969093600480935F0480915E039091CD
:100D00005F038A309105D4F00A9790935F03809334
:100D10005E0380915103909152030A96909352037F
:100D2000809351036EE170E00E942728892B31F4F3
:100D300083E090E061E070E00E94BA0482E193E019
:100D400060E00E94C30F82E193E065E041E12AE4A4
:100D500007E00E94C01082E193E061E00E94C30FAF
:100D600086E080931B0382E180931C0382E193E081
:100D700062E671E00E94AF2486E480931B036091D9
:100D8000560370E06E5F7F4F82E193E04AE050E0EF
:100D90000E949C2480915F0490916004C2978CF023
:100DA000809156038F5F809356038AE493E062E755
:100DB00071E00E94CB2582E090E061E070E00E944B
:100DC000BA040F9108950F9382E193E060E00E94CE
:100DD000C30F82E193E066E140E127E209E00E946F
:100DE000C01082E193E061E00E94C30F88E180932C
:100DF0001B0382E180931C0382E193E06BE771E0C7
:100E00000E94AF2482E193E066E140E127E20E9484
:100E1000F61084E080931B038AE280931C0382E136
:100E200093E065E871E00E94AF248CE592E065E014
:100E30000E94730F882351F08AE493E069E971E01E
:100E40000E94CB2587E792E00E94181F0F9108951A
:100E50004F925F926F927F928F929F92AF92BF92CA
:100E6000CF92DF92EF92FF920F931F9380916104D4
:100E7000909162048F5F9F4F09F0B5C080915F042D
:100E800090916004892B09F0AEC080915803909135
:100E900059036AE070E00E942728A62E80915A0329
:100EA00090915B036AE070E00E942728B62EFA2C2E
:100EB000F39482E193E06F2D4B2D0E940410482E95
:100EC000A2E0CA2ECA0C1B2D1F5F82E193E06C2D9D
:100ED000412F0E940410582EF3E0DF2EDA0C82E13D
:100EE00093E06D2D412F0E940410682E0A2D0C5F97
:100EF00082E193E0602F4B2D0E940410782EE4E0F5
:100F0000EE2EEB0C82E193E06F2D4E2D0E9404102B
:100F1000882E1E5F82E193E06C2D412F0E94041009
:100F2000982E82E193E06D2D412F0E940410C82E6F
:100F300082E193E0602F4E2D0E940410D82E1150B4
:100F400082E193E06F2D412F0E940410E82E82E190
:100F500093E0602F412F0E940410F82E80915D03D2
:100F60008B508230D0F480915C038930B0F08C30AB
:100F7000A0F41D5F82E193E06A2D412F0E940410CE
:100F8000082F85E0A80E82E193E06A2D412F0E9490
:100F9000041010E0080F111D02C000E010E0842DC5
:100FA00090E0850D911D860D911D870D911D880D79
:100FB000911D890D911D8C0D911D8D0D911D8E0D15
:100FC000911D8F0D911D800F911F892B61F08EE176
:100FD00090E0909362048093610481E090E061E08E
:100FE00070E00E94BA041F910F91FF90EF90DF9084
:100FF000CF90BF90AF909F908F907F906F905F90B9
:101000004F9008951F9312E110931C038AE0809380
:101010001B0382E193E06FE971E00E94AF2482E458
:1010200080931B036091560370E06F5F7F4F82E1F6
:1010300093E04AE050E00E949C2484E280931C03E9
:1010400082E080931B0382E193E06DEA71E00E94ED
:10105000AF2410931B038AE280931C0382E193E088
:1010600062EC71E00E94AF248CE592E060E042E027
:101070000E947D0F882369F080915603882349F0F0
:1010800081508093560384E090E061E070E00E941C
:10109000BA048CE592E062E042E00E947D0F882372
:1010A00079F0909156038091DC01981748F49F5F86
:1010B0009093560384E090E061E070E00E94BA04EF
:1010C0008CE592E065E041E00E947D0F882361F0AD
:1010D0008AE493E062E771E00E94CB2584E090E02F
:1010E00061E070E00E94BA041F9108958CE592E0DF
:1010F00060E041E00E947D0F882309F450C0809198
:101100006104909162048F5F9F4F09F048C0809105
:101110005F0490916004892B09F041C080915C03C9
:10112000815080935C0380915E0390915F030197EF
:1011300090935F0380935E0380E090E060E070E056
:101140000E94BA0480915E0390915F03C29734F4C9
:1011500083E090E061E070E00E94BA04809158035F
:10116000909159036AE070E00E942728262F2A5F99
:1011700080915A0390915B036AE070E00E942728F7
:10118000462F4F5F82E193E0622F26EC32E00E940F
:10119000DD1280915C038F3F11F410925C038CE5AB
:1011A00092E062E041E00E947D0F882309F451C083
:1011B00080916104909162048F5F9F4F09F049C054
:1011C00080915F0490916004892B09F042C0809166
:1011D0005C038F5F80935C0380915E0390915F035B
:1011E000019790935F0380935E0380E090E060E05E
:1011F00070E00E94BA0480915E0390915F03C297F1
:1012000034F483E090E061E070E00E94BA048091E1
:101210005803909159036AE070E00E942728262F16
:10122000245080915A0390915B036AE070E00E9421
:101230002728462F4F5F82E193E0622F26EC32E0B1
:101240000E94DD1280915C03853118F084E1809367
:101250005C038CE592E064E040E00E947D0F88230F
:1012600009F450C080916104909162048F5F9F4F98
:1012700009F048C080915F0490916004892B09F0C7
:1012800041C080915D03825080935D0380915E0335
:1012900090915F03019790935F0380935E0380E0DA
:1012A00090E060E070E00E94BA0480915E0390914B
:1012B0005F03C29734F483E090E061E070E00E9445
:1012C000BA0480915803909159036AE070E00E943B
:1012D0002728262F2F5F80915A0390915B036AE0A5
:1012E00070E00E942728462F4B5F82E193E0622F37
:1012F00026EC32E00E94DD1280915D038B3F10F0FE
:1013000010925D038CE592E066E00E94730F8823E3
:1013100071F082E592E06EE474E048E650E00E94ED
:101320006D188AE493E069E971E00E94CB25809111
:101330005E0390915F0397FF04C010925F031092C9
:101340005E03809161038F5F8093610390E0409121
:10135000620322E030E0241B31092817390764F4C6
:1013600080915D038F5F80935D03109261038531EF
:1013700018F084E180935D030895CF93DF9320916B
:101380006104309162048FEF2F3F3807E9F56091D7
:101390005F04709160046115710509F0B6C1809118
:1013A0005803909159030A9720915C03820F911D75
:1013B000909359038093580340915A0350915B03D3
:1013C0004A50504020915D03420F511D50935B03E2
:1013D00040935A038D50934034F08CE093E0909307
:1013E000590380935803809158039091590397FFB4
:1013F00004C0109259031092580357FF86C11092EF
:101400005B0310925A0381C1C90164E070E00E943D
:101410002728462F80915803909159036AE070E085
:101420000E942728E62FE40FEA5080915A039091FA
:101430005B036AE070E00E942728460F4A50C9010A
:1014400066EF7FEF0E9427289B01F3E0220F331FF6
:10145000FA95E1F722543D4F82E193E06E2F0E940E
:10146000DD122091610430916204809158039091C3
:1014700059036AE070E00E942728E62FC90164E062
:1014800070E00E942728E60FEA5080915A0390915D
:101490005B036AE070E00E942728462FC90164E0E0
:1014A00070E00E942728461B465FC90166EF7FEF68
:1014B0000E9427289B0173E0220F331F7A95E1F7E2
:1014C00022543D4F82E193E06E2F0E94DD12209165
:1014D00061043091620480915803909159036AE04D
:1014E00070E00E942728E62FC90164E070E00E94A6
:1014F0002728E61BE65F80915A0390915B036AE020
:1015000070E00E942728462FC90164E070E00E9425
:101510002728460F4A50C90166EF7FEF0E9427280F
:101520009B0163E0220F331F6A95E1F722543D4F80
:1015300082E193E06E2F0E94DD12209161043091D0
:101540006204C90164E070E00E942728462F41959B
:1015500080915803909159036AE070E00E94272817
:10156000E62FE40FE65F80915A0390915B036AE0F7
:1015700070E00E942728460F465FC90166EF7FEFA3
:101580000E9427289B0153E0220F331F5A95E1F751
:1015900022543D4F82E193E06E2F0E94DD120E94A3
:1015A000130676C080915C03893010F08C3018F0FF
:1015B000672B09F454C080915803909159036AE055
:1015C00070E00E942728262F80915A0390915B0398
:1015D0006AE070E00E942728462F82E193E0622FA4
:1015E0002EE932E00E94DD12809158039091590358
:1015F0006AE070E00E94272880915703C82FD0E04E
:10160000FE01E352FE4F808190E0880F991F880F02
:10161000991F68177907E4F1069686179707C4F1B2
:1016200080915A0390915B036AE070E00E94272842
:101630006A5F7F4FC951DE4F888190E0880F991F04
:10164000880F991F681779071CF180915F049091AA
:101650006004892BE9F481E08093600319C08091D4
:101660005803909159036AE070E00E942728262FC2
:1016700080915A0390915B036AE070E00E942728F2
:10168000462F82E193E0622F26E932E00E94DD12CC
:1016900082E193E060E00E94C30FE0915703F0E025
:1016A000DF01A352BE4F6C9170E0660F771F660F8B
:1016B000771FE951FE4F4081440F440F4F5F82E195
:1016C00093E02CE00E94AC1082E193E061E00E9484
:1016D000C30FE0915703F0E0DF01A352BE4F6C91BE
:1016E00070E0660F771F660F771FE951FE4F40814C
:1016F00050E0440F551F440F551F82E193E02CE04A
:101700000E94AC10DF91CF91089580915D038B50C2
:10171000823008F04DCF46CF0F9380915A039091BD
:101720005B038E3691050CF454C082E193E060E0D7
:101730000E94C30F82E193E060E040E024E506E010
:101740000E94C01082E193E061E00E94C30F1092FA
:101750001C0360915103709152036A30710514F4B7
:1017600081E501C08DE46436710514F430E001C0F8
:1017700034E093E0683E790714F420E001C024E0EF
:1017800097E26031790714F490E001C094E0831B84
:10179000821B891B80931B0382E193E04AE050E0A7
:1017A0000E949C2410921B0382E193E06FEC71E095
:1017B0000E94AF2480915E0390915F036AE070E025
:1017C0000E942728262F82E193E064E042E00E94F5
:1017D000AC100F9108952F923F924F925F926F92AB
:1017E0007F928F929F92AF92BF92CF92DF92EF92B1
:1017F000FF920F931F93DF93CF9300D000D00F92EF
:10180000CDB7DEB7309156032091DC01622F70E036
:101810006F5F7F4F832F90E00E94272880935703AC
:10182000231718F481E08093620382E193E060E083
:101830000E94C30F82E193E060E040E025E10CE00C
:101840000E94C01082E193E061E00E94C30F2091EA
:10185000570386E2289F9001112425533D4F82E1D2
:1018600093E060E040E00E94DD12AA24BB24222421
:10187000239444244A9474C1CA8282E193E06C2D7B
:101880004B810E9404108983C114D10471F0A1140A
:10189000B10421F491E0892E912C18C082E193E0EB
:1018A000652D442D0E94041009C0A114B10431F427
:1018B00001E010E081E0882E912C2BC082E193E0C2
:1018C0006A81442D0E940410882E992424E1C216B6
:1018D000D10479F0A114B10431F082E193E0632DD9
:1018E000442D0E940410C114D10419F401E010E049
:1018F00010C082E193E0652D4B810E940410082FF7
:1019000010E034E1C316D10421F4B1E0EB2EF12C48
:101910000BC082E193E0632D4B810E940410E82EFE
:10192000FF24C114D10471F08BE0A816B10419F49E
:10193000E1E0F0E018C082E193E0652D422D0E94C5
:10194000041009C0FBE0AF16B10429F421E030E037
:101950003D832C8318C082E193E06A81422D0E946E
:101960000410E82FF0E0FD83EC83F4E1CF16D104FE
:1019700051F02BE0A216B10431F082E193E0632D27
:10198000422D0E9404103981313019F060E070E07E
:10199000D0C00115110519F061E070E008C064E0E5
:1019A00070E080E090E00E94FB246E5F7F4FE114C6
:1019B000F10441F464E070E080E090E00E94FB24D8
:1019C0006A5F7F4F8114910441F464E070E080E02D
:1019D00090E00E94FB24665F7F4F8C819D81892B64
:1019E00041F464E070E080E090E00E94FB24625FDC
:1019F0007F4F81149104A9F40115110509F0EEC07F
:101A000064E070E080E090E00E94FB246E5E7F4F17
:101A1000E5C064E070E080E090E00E94FB246A5E34
:101A20007F4F0115110561F4EC81FD81EF2B41F42D
:101A300064E070E080E090E00E94FB24665E7F4FEF
:101A4000E114F10461F42C813D81232B41F464E025
:101A500070E080E090E00E94FB24625E7F4F811482
:101A6000910461F48C819D81892B41F464E070E0E4
:101A700080E090E00E94FB246E5C7F4F0115110511
:101A800059F4E114F10441F464E070E080E090E086
:101A90000E94FB246A5C7F4F8114910461F501155B
:101AA000110509F0A0C0EC81FD81EF2B09F09BC06E
:101AB00064E070E080E090E00E94FB246E5D7F4F68
:101AC00092C02C813D81232B09F091C064E070E02D
:101AD00080E090E00E94FB246A5D7F4F88C0E114A3
:101AE000F10461F464E070E080E090E00E94FB2487
:101AF000665D7F4F06C001151105D9F4E114F104AC
:101B000061F48C819D81892B41F464E070E080E078
:101B100090E00E94FB24625D7F4F892851F4012BE5
:101B200041F4EF2831F4EC81FD81EF2B11F46AE3ED
:101B300070E0F30160830894C11CD11C2CE030E0FC
:101B4000620E731E3394539434E1531609F094CE0D
:101B50000894A11CB11C239443948BE0481671F0A7
:101B6000A3E66A2EA3E07A2E6A0C7B1CCC24DD242B
:101B70003324339455245A94AB827ECE82E193E091
:101B800060E00E94C30F82E193E060E040E025E165
:101B90000CE00E94C01082E193E061E00E94C30F5C
:101BA0008AE493E06AE571E00E94CB250F900F90E4
:101BB0000F900F900F90CF91DF911F910F91FF9099
:101BC000EF90DF90CF90BF90AF909F908F907F90DD
:101BD0006F905F904F903F902F900895E114F10423
:101BE00009F01FCF16CFE114F10409F46ACF0115F3
:101BF000110509F474CF9DCF82E592E00E94B417DD
:101C0000882309F452C08AE493E06EE371E00E94F5
:101C10002525882311F00E946E058AE493E069E08F
:101C200071E00E942525882311F00E9402088AE4B1
:101C300093E062E771E00E942525882311F00E945D
:101C4000EB0B8AE493E06AE571E00E942525882386
:101C500011F00E9446058AE493E061E071E00E9481
:101C60002525882371F00E9476080E940F050E94A6
:101C700028070E94BD090E946E060E9413060E945A
:101C80008C0B8AE493E069E971E00E9425258823A2
:101C900011F00E947E058AE493E061E571E00E9404
:101CA0002525882311F00E94E30608950F931F93C2
:101CB00002E512E0C8010E94D019C80164E10E9447
:101CC000A115C80169E574E048E650E00E946D186E
:101CD000C8010E9469178AE493E069E971E00E94F3
:101CE000CB2510926A021F910F910895882319F451
:101CF0008CB5806202C08CB58F7D8CBD08959CB57B
:101D0000937F982B9CBD08952CB5382F33702C7F72
:101D1000322B3CBD2DB590E095958795959587958F
:101D200081702E7F822B8DBD08958AE061E00E9434
:101D30009D228AE061E00E945E228CB580618CBDAC
:101D40008CB580648CBD8DE061E00E945E228BE0EA
:101D500061E00E945E220895FC0181E08083089585
:101D600085E070E00E94FE2108956F927F928F922D
:101D70009F92AF92BF92CF92DF92EF92FF920F931A
:101D80001F93CF93DF93EC0189819A818C0124E02A
:101D9000000F111F2A95E1F7081B190B85E10E941E
:101DA000DC21BC01600F711F84E0769567958A95F0
:101DB000E1F77A8369838881882381F12E813F81CD
:101DC0006217730710F4B90106C0888599858617D4
:101DD000970708F4BC0100D000D080E090E040E01C
:101DE00050E0E884F98400E010E0AD80BB24CC240E
:101DF000DD246C80772488249924EDB7FEB76182B6
:101E00007282838294820E94B2246B830F900F901F
:101E10000F900F9085E070E00E94FE21DF91CF913E
:101E20001F910F91FF90EF90DF90CF90BF90AF90F8
:101E30009F908F907F906F900895FC018CE39FE0BE
:101E40009383828384E0818381E084870895CF93A4
:101E5000DF93EC018C8590E08F719070892B69F590
:101E600084E10E94DC21AA2797FDA095BA2FBC012E
:101E7000CD010E94F92626EE3FE34EEC50E40E948D
:101E800085270E94CB269B01AC017B836A83611569
:101E9000710589F084E08983B901FE0120E0848125
:101EA00095816817790710F429830AC02F5F32964D
:101EB0002430A9F702C08FEF89838C858F5F8C87D0
:101EC000DF91CF910895FC0188E0808389E08183D0
:101ED00087E0828386E0838384E0848382E0858355
:101EE00081E18683089520E0FC01E60FF11D8781E2
:101EF000813009F421E0822F0895E62FF0E042308E
:101F000040F420E0E80FF91F878181508E3F88F46C
:101F10000FC0E80FF91F87818F3F11F420E009C03F
:101F200020E090E0642F70E00E941328019709F4EC
:101F300021E0822F08950F931F93CF93DF93EC013D
:101F400010E00FEF888162E00E945E2288810E948B
:101F5000F1222F81892B19F42F5F2F8307C02223B1
:101F600049F02F3F11F41F8201C00F83888160E088
:101F70000E945E221F5F2196173021F7DF91CF91DB
:101F80001F910F910895FC01678F60A30895FC01D4
:101F9000678F40A30895FC016435A8F547FD33C061
:101FA00040338CF5878D942F95959595959577274A
:101FB00067FD70954770882399F0E4E59E02F00173
:101FC0001124E60FF71FED59FB4F81E090E002C0AE
:101FD000880F991F4A95E2F72081282B20830895C6
:101FE000E4E59E02F0011124E60FF71FED59FB4FC7
:101FF00081E090E002C0880F991F4A95E2F7809532
:102000002081282320830895742F643530F547FDFF
:1020100024C0403314F5842F85958595859599279F
:1020200087FD9095462F552747FD509524E530E0D4
:10203000829FF001839FF00D929FF00D1124E40F19
:10204000F51FED59FB4F808190E0777002C09595A8
:1020500087957A95E2F78170089580E00895AF92B0
:10206000BF92CF92DF92EF92FF920F931F93CF9385
:10207000DF93EC01162FF42EE22EAA24402F5527D1
:1020800047FD50958F2D992787FD9095481B590B3B
:1020900057FF03C0509541955F4F2E2D332727FDE5
:1020A0003095812F992787FD9095281B390B37FF95
:1020B00003C0309521953F4F2417350744F4AA24D7
:1020C000A3948F2DF12E182F802F0E2DE82EE116C0
:1020D00034F48E2DE12E182F802F0F2DF82EDE2CAC
:1020E000D11A202F332727FD30958F2D992787FD73
:1020F0009095281B390B37FF03C0309521953F4F32
:10210000B22EF0161CF0CC24CA9402C0CC24C39486
:102110008D2DD7FC8F5F082F059511C0AA2021F0C7
:10212000CE016F2D412F03C0CE01612F4F2D0E9494
:10213000CB0F0B1907FF02C0FC0C0D0D1F5FE11642
:102140006CF7DF91CF911F910F91FF90EF90DF908F
:10215000CF90BF90AF9008950F93042F322F262F6A
:102160002150230F0E942F100F9108950F93362FA7
:10217000042F0150020F232F0E942F100F9108955A
:102180009F92AF92BF92CF92DF92EF92FF920F9306
:102190001F93CF93DF936C01B62E942EA02EC0E038
:1021A000D0E0E62EFF24E7FCF094022F112707FD74
:1021B00010950E0D1F1D06C0C601492D2A2D0E9427
:1021C000B61021966B2D6C0FCE018E0D9F1D8017C2
:1021D000910794F3DF91CF911F910F91FF90EF90B2
:1021E000DF90CF90BF90AF909F900895CF92DF92F5
:1021F000EF92FF920F931F937C01162FD42EC22EC5
:102200000E94AC104D2D4150400FC701612F2C2D65
:102210000E94AC10C701612F4D2D202F0E94B610D7
:1022200011501C0DC701612F4D2D202F0E94B6109B
:102230001F910F91FF90EF90DF90CF9008952F9214
:102240003F925F926F927F928F929F92AF92BF92D6
:10225000CF92DF92EF92FF920F931F93DF93CF9372
:1022600000D000D000D0CDB7DEB79E838D83C62EC0
:10227000D42EEE24E394E21A8EEF289F502C1124E2
:10228000842E8A94962E9A94A42EA394B62EB39458
:10229000F22E662423E0722E10E0C8018470907044
:1022A0009A838983F801E270F070FC83EB8398E0F5
:1022B000292E312C202231220170107054C0E7FCED
:1022C00004C0FA94F2E05F0EE50C639489819A8170
:1022D000892B71F04F2D4D0D8D819E816B2D0E94AC
:1022E000CB0F6F2D6C0D8D819E814A2D0E94CB0FDF
:1022F000EB81FC81EF2B71F04D2D4F198D819E816B
:102300006B2D0E94CB0F6F2D6C0D8D819E81482D02
:102310000E94CB0F2114310471F06C2D6F198D8147
:102320009E814A2D0E94CB0F4F2D4D0D8D819E8198
:10233000692D0E94CB0F0115110571F06C2D6F19DD
:102340008D819E81482D0E94CB0F4D2D4F198D817F
:102350009E81692D0E94CB0FE70CF2E07F0E8A94DC
:102360009A94A394B3946F140CF4A9CF26960FB645
:10237000F894DEBF0FBECDBFCF91DF911F910F91BB
:10238000FF90EF90DF90CF90BF90AF909F908F9095
:102390007F906F905F903F902F9008954F925F9243
:1023A0006F927F928F929F92AF92BF92CF92DF9265
:1023B000EF92FF920F931F93CF93DF93EC01A62E22
:1023C000742E9E2DFF24F394F21A8EEF289F802CFA
:1023D0001124B42EBA9453E0C52ECE0CE22EDD2487
:1023E00043E0942E10E031E0432E512C4022512244
:1023F000692E63940270107034C0F7FC04C0EA9434
:1024000082E0880EF80CD3944114510489F06D2DAC
:102410006A0D472D4E192E2D220F260DCE010E943A
:10242000B6106E2D6A0DCE014B2D2C2D0E94B610CC
:102430000115110589F06A2D6D19472D4E192E2DA4
:10244000220F260DCE010E94B6106A2D6E19CE0104
:102450004B2D2C2D0E94B610F90C82E0980EBA94E8
:10246000C80EDE1454F2DF91CF911F910F91FF90AF
:10247000EF90DF90CF90BF90AF909F908F907F9024
:102480006F905F904F9008957F928F929F92AF923E
:10249000BF92CF92DF92EF92FF920F931F936C0146
:1024A000962EA42EF22E7E2C760E1EEFE19E102D7F
:1024B0001124812E820E672D282D0E94AC10B02E83
:1024C000BA0CBA94C601672D4B2D282D0E94AC1072
:1024D000AE0C100FC601692D4A2D212F0E94B61097
:1024E000F90CFA94C6016F2D4A2D212F0E94B610C7
:1024F000C601672D4A2D2E2D01E00E941F11FE18E6
:10250000C6016F2D4A2D2E2D02E00E941F11BE180C
:10251000C6016F2D4B2D2E2D04E00E941F11C60108
:10252000672D4B2D2E2D08E00E941F111F910F913A
:10253000FF90EF90DF90CF90BF90AF909F908F90E3
:102540007F9008958F929F92AF92BF92CF92DF9229
:10255000EF92FF920F931F936C01162FA42E922ED1
:10256000F02EBE2C8E2C860E2EEFE29EE02C112437
:102570002E2D290D682D0E94C010AB0CFA94FE0C74
:102580001150190D1B19C601612F4A2D2B2D01E089
:10259000EF2C0E94CE11C601682D4A2D2B2D02E092
:1025A0000E94CE111F910F91FF90EF90DF90CF907E
:1025B000BF90AF909F908F9008953F924F925F92FF
:1025C0006F927F928F929F92AF92BF92CF92DF9243
:1025D000EF92FF920F931F93CF93DF934C01362E10
:1025E000442EF901A490319654906F010894C11CB7
:1025F000D11C8A2D992787FD9095079668E070E099
:102600000E942728E62EFF24E7FCF09400E0C0E0BB
:10261000D0E060E8662E712C26C0E12FE595E595A7
:10262000E595FF27E7FDF095EC0FFD1FEC0DFD1D77
:10263000E4912E2F30E0812F8770A30102C05595C1
:1026400047958A95E2F724233523232B31F0612F18
:10265000630DC4014B2D0E94CB0F1F5F1A15ECF2C6
:102660000F5FCE0DDF1D051524F410E0B02EB40C65
:10267000F5CFDF91CF911F910F91FF90EF90DF90F9
:10268000CF90BF90AF909F908F907F906F905F9012
:102690004F903F9008953F924F925F926F927F923A
:1026A0008F929F92AF92BF92CF92DF92EF92FF9262
:1026B0000F931F93CF93DF93EC01862EA42E422F0E
:1026C000102F3F8C23E526170CF4ABC03FE23A15E0
:1026D0000CF4A7C0C02EDD248C8190E001979C01F2
:1026E000C29EC001C39E900DD29E900D1124262F34
:1026F000332727FD3095820F931F181619060CF00B
:1027000090C08D8190E09C01C29EC001C39E900D3F
:10271000D29E900D11242A2D332727FD3095820F4C
:10272000931F181619060CF07CC09924442E5524CA
:102730006DC09C01215030404217530711F460E0F6
:102740000EC0429EC001439E900D529E900D1124DA
:10275000840F951FED8DFE8DE80FF91F64914C9D40
:10276000C0014D9D900D5C9D900D1124682C680E4C
:10277000BB24792C780C3FC0E62EFF2460FF19C0E3
:10278000113039F44B2D4A0DCE01672D0E94CB0F2D
:102790002EC02C9DC0012D9D900D3C9D900D1124AF
:1027A0004A2D480FCE01662D212F012F0E94C01007
:1027B0001EC098A18F8D9817D1F09F8F113039F4DA
:1027C0004B2D4A0DCE01672D0E94CB0F0FC02C9DC3
:1027D000C0012D9D900D3C9D900D11244A2D480F58
:1027E000CE01662D212F012F0E94C0103F8EF5943F
:1027F000E7946E2DB3942B2D332727FD30958D81D3
:1028000090E0281739070CF4B7CF9394492D55273A
:1028100047FD50958C8190E0481759070CF489CFFB
:102820003F8EDF91CF911F910F91FF90EF90DF903E
:10283000CF90BF90AF909F908F907F906F905F9060
:102840004F903F9008950F93CF93DF93EC01262F85
:102850006A3049F48D819885899F802D11249A854D
:10286000980F9A8726C06D3029F169854A850885B9
:102870000E944B139C816885969F402D1124898569
:10288000480F49878F818823A9F0552747FD509528
:10289000699F9001112484E590E0821B930B8417BB
:1028A000950744F49D81699F902D11248A85890F95
:1028B0008A87198681E090E0DF91CF910F9108958A
:1028C0001F93CF93DF93EC01162FF8948E8560E071
:1028D0000E949D228F8518161CF460E00E949D22A4
:1028E0001EBD0DB407FEFDCF8EB58F8518161CF4E6
:1028F00061E00E949D227894DF91CF911F9108950D
:10290000FF920F931F93CF93DF93EC01FF2400E01E
:1029100010E06F2D6064CE010E946014CE0160E86B
:102920000E9460148E8561E00E949D228F8518169A
:102930001CF460E00E949D22F801ED59FB4F90E0ED
:1029400080818EBD0DB407FEFDCF8EB59F5F3196A1
:102950009435B1F78F8518161CF461E00E949D2212
:10296000F3940C5A1F4F86E0F81699F6CE0160E4F6
:102970000E946014DF91CF911F910F91FF900895F5
:10298000CF93DF93DC0188EF91E0E3E6F4E0EF0121
:102990009C01199221503040E1F719961C92199729
:1029A0001A961C92DF91CF910895EF920F93CF93D7
:1029B000DF93EC014D876C872E87E88A0F8781E0D3
:1029C00088878F8F18A28F83E4E6F4E084918F5F6D
:1029D0008C83319684918F5F8D833196FE8FED8F3E
:1029E0000E94950E81E00E94760E85E00E94840E82
:1029F0008CE00E947F0E8D8561E00E945E228C85B6
:102A000061E00E945E228E8561E00E945E228889DC
:102A100018161CF461E00E945E228F8518161CF4C3
:102A200061E00E945E22888918166CF460E00E94C2
:102A30009D226AE070E080E090E00E944821888951
:102A400061E00E949D22EC852E2F332727FD3095D3
:102A5000F901E257F84FE491F0E0EE0FFF1FE6585E
:102A6000F84F859194919C8B8B8B2E55384FF901A3
:102A700084918A8FED852E2F332727FD3095F9011C
:102A8000E257F84FE491F0E0EE0FFF1FE658F84FE1
:102A9000859194919A8B898B2E55384FF9018491A9
:102AA000898FEF852E2F332727FD3095F901E257C7
:102AB000F84FE491F0E0EE0FFF1FE658F84F8591D4
:102AC00094919E8B8D8B2E55384FF90184918B8F6D
:102AD000EE852E2F332727FD3095F901E257F84F69
:102AE000E491F0E0EE0FFF1FE658F84F85919491C6
:102AF000988F8F8B2E55384FF90184918C8FCE0192
:102B000061E20E946014CE0164E10E9460148B8532
:102B100087FF02C08FE78B876B856068CE010E94BC
:102B20006014CE0160E20E946014CE016CE00E944D
:102B30006014CE010E948014DF91CF910F91EF902D
:102B40000895FC01262FE051FF4F88EE93E070E0DE
:102B50000E9427286083E05FF040822F64E10E949A
:102B6000072885AB0895CF93DF93DC01E0E8FFE60B
:102B700085919491ED01C553DF4FAD014F515F4FEA
:102B80008150904C09F04EC0E6E9FFE6E491E883FD
:102B9000E7E9FFE6E4911496EC931497E8E9FFE681
:102BA000E4911596EC931597E9E9FFE685919491E8
:102BB00017969C938E931697EBE9FFE68591949177
:102BC00019969C938E931897EDE9FFE6E491D796BA
:102BD000EC93D797EEE9FFE6E491D696EC93D6977F
:102BE000EFE9FFE6E491EA01E883E0EAFFE6859198
:102BF00094915D969C938E935C97E2EAFFE68591B3
:102C000094915F969C938E935E97E4EAFFE685919C
:102C1000949191969C938E939097E6EAFFE6859126
:102C2000949132C08CE3888314961C9214972FEFF2
:102C300015962C93159780E293E017969C938E93AC
:102C4000169784ED93E019969C938E93189781E0E4
:102C5000D7968C93D797D6968C93D697FA012083E4
:102C60008CEA9DE05D969C938E935C978EED9DE043
:102C70005F969C938E935E9784E79EE091969C93DB
:102C80008E9390978CE39FE093969C938E9392976C
:102C9000DF91CF910895EF92FF920F931F93CF93FF
:102CA000DF937C018C0100541F4FC8010E94C014A7
:102CB000C8016BE076E00E947D23C8010E94801469
:102CC00083E00E94840E81ED91E0EEEFFFE3099531
:102CD00086EC90E0E80EF91EF7011082C80166EE5E
:102CE00075E00E94C823C8010E948014E701CC5BF4
:102CF000D040CE010E949B0FCE0164E00E94730F72
:102D0000882339F462E370E080E090E00E9448217B
:102D1000F0CFDF91CF911F910F91FF90EF90089529
:102D20000F931F93CF93DF93EC018C0100541F4F3F
:102D3000C80161E040E00E94C70FFE01E753FF4F6A
:102D4000CC53DF4F85E59881891B808326961882B6
:102D5000CA5CD040698D613081F1613028F0888D86
:102D6000653008F043C03DC0CE0185960E942C1B03
:102D7000CE0160E00E94B00EC8010E94C014C8538A
:102D8000DF4F81E08883C80163E376E00E947D2302
:102D9000C8010E94801483B7817F846083BF83B79A
:102DA000816083BF83B7816083BF889583B78E7F3F
:102DB00083BF83B78E7F83BF1FC0CE51DF4F888113
:102DC0009981AA81BB818F709070A070B0700897B4
:102DD000A105B10518F4C80167E00CC0C80168E797
:102DE00009C0882349F06B5FC80104C0882321F023
:102DF000C8016FE20E94A023DF91CF911F910F9134
:102E00000895AF92BF92CF92DF92EF92FF920F930D
:102E10001F93CF93DF93EC01C950DF4F8881C75FC9
:102E2000D040882309F44AC08C3010F010E002C072
:102E30001CE0181BC853DF4F81E08883C85CD0407A
:102E400060ECC62ED12CCC0EDD1EC60160E00E94C7
:102E5000C30F55ECA52EB12CAC0EBD1EF5010081A3
:102E60004DE2F42E4F2D401B410F0D5FC60160E077
:102E700024E533E0E32E0E94A212C60161E00E9425
:102E8000C30FF5010081F01AF10E0D5FC60160E07D
:102E90004F2D24E50E944412C753DF4F84E08993ED
:102EA000F5018081181B115D1883AB9669917991AA
:102EB000C6010E947D23888181508883DF91CF9154
:102EC0001F910F91FF90EF90DF90CF90BF90AF9048
:102ED00008954F925F926F927F928F929F92AF92DE
:102EE000BF92CF92DF92EF92FF920F931F932C012C
:102EF000FC01628C738C60947094882499240E94E5
:102F000022215B016C010E9422217B018C01F201D4
:102F1000418052800E942221460E571EA094B094F8
:102F2000C094D094E094F09400951095C601B5013A
:102F3000A80197010E94E827A40193010E94E827B5
:102F4000460E571EC2010E941D251F910F91FF9032
:102F5000EF90DF90CF90BF90AF909F908F907F9039
:102F60006F905F904F900895AF92BF92CF92DF9293
:102F7000EF92FF920F931F93CF93DF93EC01E1EF5A
:102F8000AE2EB12CA80EB91EF501E080F1800281B1
:102F900013810E941421E61AF70A080B190B70EF2F
:102FA000C72ED12CCC0EDD1EF601808190E0A0E072
:102FB000B0E08E159F05A007B10708F081C08E0113
:102FC00004511F4FF80180819181A281B381009744
:102FD000A105B10509F474C00E941421F6012081F5
:102FE000620F711D811D911DF501608371838283C4
:102FF0009383FE01EE51FF4F80819181A281B381C5
:103000000196A11DB11D80839183A283B383F80132
:1030100010821182128213820E942221C851DF4F36
:10302000688379838A839B83C85ED040CE010E94E7
:10303000B50ECE010A960E949B0FCE0148960E94C3
:10304000270F81E032C08E010B5D1F4FC8010E9427
:10305000AF1BC8010E94931CC8010E940F1ECE0125
:103060000E940117CE010E9490168E0100541F4F3E
:10307000C8010E948014CA53DF4F8881C65CD040CB
:10308000882319F4C8010E94C0140E942221C4514F
:10309000DF4F688379838A839B83249728813981D2
:1030A000621B730B7A936A9380E0DF91CF911F913B
:1030B0000F91FF90EF90DF90CF90BF90AF90089569
:1030C000C451DF4F88819981AA81BB81CC5ED040F9
:1030D0000097A105B10541F7B6CF2F923F924F92CD
:1030E0005F926F927F928F929F92AF92BF92CF9298
:1030F000DF92EF92FF920F931F93DF93CF93CDB7A1
:10310000DEB72B970FB6F894DEBF0FBECDBF9B87FF
:103110008A877A8369835C834B838C010F511F4FAD
:10312000F8018081882309F422C18A859B85885310
:103130009F4F9B878A8781E0EA85FB858083129277
:103140001292E65CF040FB87EA87108E90ECE92E45
:10315000F12CEE0EFF1EC70161E00E94C30F8AE052
:10316000282E312C8A859B85280E391EB5E26B2EC0
:10317000712C680E791EE981FA81F491FD83A9EC26
:103180008A2E912C880E991EFAECCF2ED12CC80EC7
:10319000D91EE4EC4E2E512C480E591E8B539F4FD6
:1031A0009F838E8372EEA72EB12C8A859B85A80EF5
:1031B000B91E198708878A859B850E94B4178823C2
:1031C000D1F39D81992311F410E003C0EE81FF81BA
:1031D0001081C70160E040E02FE736E00E94DD1279
:1031E0008B819C81892B41F0145FC70160E0412FE6
:1031F0002B813C810E94DD12F40110828CE0F601EB
:103200008083C70169817A810E947D23F201208138
:1032100030E0C901880F991F820F931F9095819507
:103220009F4F8D5AF4018083EE81FF81208130E031
:10323000C901880F991F820F931F909581959F4F09
:10324000835DF6018083F501808184FF04C0C7019E
:103250006FEF76E003C0C7016BEF76E00E94C823F2
:10326000F201208130E0C901880F991F820F931F5E
:10327000909581959F4F8D5AF4018083F60180814E
:103280008F5F8083EA85FB8586A9882321F0C701AB
:1032900067EF76E003C0C70163EF76E00E94C823C2
:1032A000F201808190E09C01220F331F280F391F0B
:1032B000309521953F4F2D5AF4012083F6018081EE
:1032C0008F5F8083C7016FEE76E00E94C823C10143
:1032D00065E00E94730F882351F0EA85FB8566A99B
:1032E0006F5FC3010E94241FC3010E941E1FC10102
:1032F00064E00E94730F882399F4E885F985608162
:10330000262F30E040E050E0F50180819181A281DC
:10331000B38182179307A407B50708F16F3FF9F04F
:103320008A859B858F519F4F9B878A878FEFEA8580
:10333000FB858083E15EF040FB87EA87C30160E0A4
:103340000E941C1BC3010E94181F81E0EA85FB85B7
:10335000808F0DC08A859B850E944B162CCFC101A2
:1033600066E00E94730F882309F425CFF3CF2B96D4
:103370000FB6F894DEBF0FBECDBFCF91DF911F9186
:103380000F91FF90EF90DF90CF90BF90AF909F9004
:103390008F907F906F905F904F903F902F90089507
:1033A000AF92BF92CF92DF92EF920F93CF93DF93C2
:1033B0006C0180EF90E0C80ED91E82E3F601808395
:1033C00081E090E0A0E0B0E0B293A2939293829368
:1033D0006F0185EF9FEFC80ED91E8FEFF601808336
:1033E0008FE19FEFC80ED91EC6010E94B315C6011A
:1033F0000E94AC0EC6016FEF0E94B00E4AE0A42EF0
:10340000B12CAC0CBD1CC5010E94630FC5010E940C
:103410009B0FC60148960E941D0FC60180549F4F06
:103420006DE04BE020E10FE03EE0E32E0E94D5147A
:10343000E601A596CE010E94311FC50165E00E94FC
:10344000730F882329F0CE0160E00E94241F18C06A
:10345000CE0165E077E040E00E94411BCE0165E0CF
:1034600077E041E00E94411BCE0165E077E042E059
:103470000E94411BCE0165E077E043E00E94411BC2
:10348000DF91CF910F91EF90DF90CF90BF90AF90F1
:1034900008950F93CF93DF93DC01043008F05AC0F6
:1034A000623009F443C0633030F4662359F0613070
:1034B00009F050C00DC0633009F43EC0643009F01B
:1034C00049C040C0A00FB11DA15BBF4F4C9342C08B
:1034D000602F70E0EB01CC0FDD1FC80FD91F842FC8
:1034E00090E0880F991F2BA93CA9280F391FF901DB
:1034F00085919491CD58DF4F99838883FC01459144
:103500005491042FFD01E60FF71FE558FF4F40834C
:10351000252F3327842F90E02817390708F4052F2B
:10352000A60FB71FA158BF4F0C9314C0FC01E00FAA
:10353000F11DE55AFF4F0BC0FC01E00FF11DED59E5
:10354000FF4F05C0FC01E00FF11DE559FF4F40831F
:1035500034962083DF91CF910F910895CF93DF931D
:10356000EC012430F0F4A22FB0E0FC01EA0FFB1FC5
:10357000E95BFF4F608334964083E05CFF4F10822D
:10358000CD01880F991FC80FD91FCD57DF4F198262
:103590001882F89781E08083A15AB94F8C933496B2
:1035A0001082DF91CF910895CF93DF93EC016430C7
:1035B00008F03FC0A62FB0E0FC01EA0FFB1FED5A58
:1035C000FF4F108238971082CD01880F991FC80FC6
:1035D000D91FCD57DF4F198218823C961082FD010A
:1035E000E559F94F1082FD01E959F94F1082A15AAE
:1035F000B94F1C9280915F06882311F490E002C0BD
:1036000090916B0680916006882319F080916C067A
:10361000980F80916106882319F080916D06980FAC
:1036200080916206882319F080916E06980F90931E
:10363000B400DF91CF9108951F93CF93DF93EC01F6
:10364000162F643028F40E94D41AC10FD11D1C8299
:10365000DF91CF911F9108950F931F938C0160E02C
:103660000E941C1BC80161E00E941C1BC80162E093
:103670000E941C1BC80163E00E941C1B1F910F913C
:103680000895EF92FF921F93CF93DF93EC017B019C
:10369000142F4430F0F4642F0E941C1B812F90E003
:1036A000FC01EE0FFF1FEC0FFD1FF4A6E3A6FF9633
:1036B00011821082FE01E80FF91F81E08483E15B33
:1036C000FF4F89E080833C961082389610823896AE
:1036D0001082DF91CF911F91FF90EF9008951F937B
:1036E000CF93DF93AC01162F6430A8F5262F30E07E
:1036F000EC01C20FD31F8881882369F18C81882354
:1037000051F5D901AA0FBB1FA40FB51F8B8D90E0F7
:10371000880F991F5396ED91FC915497E80FF91F6C
:10372000859194912FEF8F3F920711F4188213C067
:103730009FA390E0880F991F5F96ED91FC91909761
:10374000E80FF91F65917491CA01412F0E94411B36
:103750008B8D8F5F8B8FDF91CF911F9108950F938A
:103760001F938C0160E00E946F1BC80161E00E9402
:103770006F1BC80162E00E946F1BC80163E00E94DA
:103780006F1B1F910F9108956F927F929F92AF923E
:10379000BF92CF92DF92EF92FF920F931F93CF933E
:1037A000DF937C01962E23E0261708F4AEC0C62EC8
:1037B000DD24DC01AC0DBD1D14968C91149788237B
:1037C00009F4A3C0A55BBF4F8C91AB54B0408823D4
:1037D00009F09BC05601AA0CBB1CAE0CBF1C850196
:1037E000015C1F4FE801E881F981EE0FFF1FE50141
:1037F0004BA55CA5E40FF51F2591349121153105EA
:1038000009F047C0DB968C91DB97813039F4F801E1
:1038100011821082FA01259134913BC014961C92BA
:1038200014978C91882381F0C7010E946F1BD801E7
:103830008D919C91880F991FE501EBA5FCA5E80FE0
:10384000F91F2591349125C0C7010E94D41A5DC08B
:10385000E6E036952795EA95E1F76F70422F4F71B4
:1038600075E0369527957A95E1F72051C701092D26
:103870000E94491A88819981019699838883880FCB
:10388000991FD501ED91FC91E80FF91F2591349115
:103890000DC03601660C771CC701860D971DEC0123
:1038A000EF964BE2A42EB12CA80EB91EB901769565
:1038B00067957695679520FDCBCFF701EC0DFD1D43
:1038C000E95BFF4F862F8F73808334963083E05CF3
:1038D000FF4F1082D701A60DB71DAD57BF4F1196F0
:1038E0001C921E92F89781E08083CFE5D6E0CC0E43
:1038F000DD1EE601888334961082A454B0408D9179
:103900009C91119701968D939C93DF91CF911F917C
:103910000F91FF90EF90DF90CF90BF90AF909F906E
:103920007F906F9008950F931F938C0160E00E9429
:10393000C41BC80161E00E94C41BC80162E00E9470
:10394000C41BC80163E00E94C41B1F910F9108951E
:10395000DF92EF92FF920F931F93CF93DF937C013F
:10396000D62E43E0461708F452C1062F10E0DC01C2
:10397000A00FB11FAD5ABF4F8C91A355B040882303
:1039800009F445C1FD01E55BFF4F8081882321F4E7
:10399000C7010E94D41A3BC181508083BD01655785
:1039A0007F4FFB018081882309F052C0F801EE0FA0
:1039B000FF1FEE0DFF1DEF01CD57DF4F888199816D
:1039C0000196880F991FED58FF4F0190F081E02D6F
:1039D000E80FF91F25913491A157BF4F822F8770AF
:1039E0008C93A901F3E056954795FA95E1F7CA0142
:1039F000969587951496232F3327269526952C93F5
:103A00008F73F7012089829F802D1124FB01808311
:103A1000F801E159F94F41704083888199810196FD
:103A20009983888358972C91AB57B04030E0821728
:103A3000930770F0A158BF4F8C91882329F0281B61
:103A400031093983288304C0C7016D2D0E94D41A1F
:103A5000E701C00FD11FFE01E557FF4F8081815064
:103A60008083FE01E95AFF4F90819F5F9083FE01A2
:103A7000ED56FF4FC95BDF4FE0818881C754D040CE
:103A8000E80F8FA1E80FE887CD59DF4F6881C35653
:103A9000D040662389F0892F992787FD909570E0A3
:103AA0000E942728C959DF4F8881C756D040869F7A
:103AB000802D11248E0F8887F701E00FF11F80857C
:103AC00090E0CB966BE370E00E9427288087E15B53
:103AD000FF4F2081EF54F0402487E55AFF4F60816B
:103AE000EB55F0406623A1F0E95AFF4F808177271C
:103AF00067FD7095992787FD90950E942728389635
:103B00008081EF55F040869F802D1124820F84879D
:103B1000F701E00FF11FE559FF4F6081EB56F040D0
:103B20006623C1F0E95AFF4F8081992787FD909560
:103B300070E00E942728CB0162E070E00E942728F5
:103B400078969081EF56F040899F802D11249485BE
:103B5000890F8487F701E00FF11F84858A300CF00C
:103B600089E0F701E00FF11F87FD80E08487F7010E
:103B7000E00FF11FE95BFF4F8081E754F0408F3386
:103B800009F41486F894A701400F511FDA01189622
:103B9000EC91F0E0E75DF84FE491D801AD59B94FF1
:103BA000EC93FA012485332727FD309549565F4F62
:103BB000DA018C9190E0F901E89F9001E99F300DC6
:103BC000F89F300D1124D70151968C9190E0F901A6
:103BD000E89F9001E99F300DF89F300D1124485067
:103BE0005040DA018C91992787FD9095FC012E9F1A
:103BF000C0012F9F900D3E9F900D1124F801E959AF
:103C0000F94F80830559194FD8018C937894DF912F
:103C1000CF911F910F91FF90EF90DF9008950F9338
:103C20001F938C0160E00E94A81CC80161E00E9403
:103C3000A81CC80162E00E94A81CC80163E00E94A1
:103C4000A81C1F910F91089560916706662341F1AA
:103C500080915B068F5F80935B0690916306891766
:103C6000F8F090E080915F06882309F491E090934A
:103C70005F0610925B0680916F06882379F0809131
:103C8000F10123E4829FC0011124895B8093F1013B
:103C900090E070E00E94132880936B0621E001C041
:103CA00020E060916806662339F180915C068F5FA1
:103CB00080935C06909164068917F0F090E0809103
:103CC0006006882309F491E09093600610925C06E8
:103CD00080917006882379F08091F10123E4829F1E
:103CE000C0011124895B8093F10190E070E00E9493
:103CF000132880936C0621E060916906662339F1F0
:103D000080915D068F5F80935D06909165068917AF
:103D1000F0F090E080916106882309F491E090939F
:103D2000610610925D0680917106882379F080917A
:103D3000F10123E4829FC0011124895B8093F1018A
:103D400090E070E00E94132880936D0621E060915E
:103D50006A06662339F180915E068F5F80935E0666
:103D6000909166068917F0F090E0809162068823B2
:103D700009F491E09093620610925E0680917206BB
:103D8000882391F08091F10123E4829FC0011124E6
:103D9000895B8093F10190E070E00E94132880938A
:103DA0006E0602C02223F9F080915F06882311F489
:103DB00090E002C090916B0680916006882319F014
:103DC00080916C06980F80916106882319F080918C
:103DD0006D06980F80916206882319F080916E0617
:103DE000980F9093B40008951F920F920FB60F9200
:103DF00011242F933F934F935F936F937F938F93F0
:103E00009F93AF93BF93EF93FF930E94241EFF9164
:103E1000EF91BF91AF919F918F917F916F915F9142
:103E20004F913F912F910F900FBE0F901F901895BB
:103E300061E277E040E00E94411B089563E177E092
:103E400040E00E94411B0895FC01862F628970E0CA
:103E50006F5F7F4F992787FD90950E942728818B60
:103E600008959F92AF92BF92CF92DF92EF92FF920E
:103E70000F931F93CF93DF93EC0181E0888B67E969
